S020000064656D6F70726F675F6F6C696D6578696E6F5F73746D33322E737265635C
S3150800800018080020298E00086D8E0008718E000859
S31508008010758E0008798E00087D8E00080000000025
S31508008020000000000000000000000000818E00082B
S31508008030858E000800000000898E0008F38C000871
S315080080408D8E0008918E0008958E0008998E00087E
S315080080509D8E0008A18E0008A58E0008A98E00082E
S31508008060AD8E0008B18E0008B58E0008B98E0008DE
S31508008070BD8E0008C18E0008C58E0008C98E00088E
S31508008080CD8E0008D18E0008D58E0008D98E00083E
S31508008090DD8E0008E18E0008E58E0008E98E0008EE
S315080080A0ED8E0008F18E0008F58E0008F98E00089E
S315080080B0FD8E0008018F0008058F0008098F00084B
S315080080C00D8F0008118F0008158F0008198F0008FA
S315080080D01D8F0008218F0008258F0008298F0008AA
S315080080E02D8F0008318F0008358F0008EE11AA552C
S315080080F02DE9FC41040000202078C0076BD5DFF885
S315080081009405016811F00C01042907D0016811F0E3
S315080081100C0108290CD10068C00309D5DFF87005E1
S315080081200068800357D56068002854D10120B3E160
S315080081306068B0F5803F06D1DFF85405016851F450
S315080081408031016026E0606800280AD1DFF8400522
S31508008150016831F480310160016831F480210160E1
S3150800816018E06068B0F5A02F0AD1DFF82405016889
S3150800817051F480210160016851F48031016009E001
S31508008180DFF80C05016831F480310160016831F4CB
S3150800819080210160606800280ED000F099FA050079
S315080081A0DFF8EC040068800315D400F091FA401B50
S315080081B06528F5D303206FE100F08AFA0500DFF899
S315080081C0D0040068800306D500F082FA401B6528B3
S315080081D0F5D3032060E1207880071ED5DFF8B404C4
S315080081E0016811F00C0F07D0016811F00C0108297D
S315080081F02CD10068C00329D4DFF8940401688907E4
S3150800820004D52169012901D0012045E1016831F031
S31508008210F801626951EAC20101602078000749D570
S31508008220A069002871D00120DFF87814086000F0F2
S315080082304FFA0500DFF868040068800737D400F0B5
S3150800824047FA401B0328F5D3032025E120690028B7
S315080082501AD00120DFF85014086000F039FA05003A
S31508008260DFF82C040168890706D400F031FA401BB0
S315080082700328F5D303200FE1016831F0F80162699C
S3150800828051EAC2010160C8E70020DFF81C14086043
S3150800829000F01EFA0500DFF8F80300688007BCD571
S315080082A000F016FA401B0328F5D30320F4E001205A
S315080082B000F0DAF92078400740F196800026DFF8CA
S315080082C0EC532868C00009D4286850F0805028600C
S315080082D0286810F08050009000980126DFF8D073C7
S315080082E03868C00524D4386850F48070386000F0C7
S315080082F0EFF980463868C0051AD400F0E9F9B0EB02
S3150800830008006528F6D30320C6E00020DFF894139A
S31508008310086000F0DDF90500DFF8840300688007CF
S31508008320C8D500F0D5F9401B0328F5D30320B3E0E0
S31508008330E068012806D1DFF87C03016851F00101E5
S31508008340016025E0E06800280AD1DFF868030168C3
S31508008350490849000160016831F00401016017E02D
S31508008360E06805280AD1DFF84C03016851F00401DA
S315080083700160016851F00101016009E0DFF834038A
S315080083800168490849000160016831F0040101608B
S31508008390E068002810D000F09BF90700DFF8140306
S315080083A00068800719D400F093F9C01B41F289319F
S315080083B08842F3D303206FE000F08AF90700DFF85C
S315080083C0F4020068800708D500F082F9C01B41F264
S315080083D089318842F3D303205EE0F6B2012E03D139
S315080083E0286830F080502860E069002853D0DFF80C
S315080083F0A462306810F00C0008284AD0E069022808
S3150800840034D1DFF8B4720020386000F061F9804694
S31508008410DFF87C522868800107D500F059F9B0EBDF
S3150800842008000328F4D3032036E0206AB0F5803F1D
S3150800843005D1316831F40031A068014331603168F3
S3150800844031F47411206A0143606A014331600120E6
S31508008450386000F03DF90400286880011BD400F05C
S3150800846037F9001B0328F7D3032015E00020DFF8AF
S315080084704812086000F02CF90400DFF814020068BE
S31508008480800108D500F024F9001B0328F5D3032042
S3150800849002E0012000E00020BDE8F6812DE9F04168
S315080084A004000D000020DFF81462306810F00700A1
S315080084B0A8420BD23068C008C00028433060306834
S315080084C010F00700A84201D0012097E02078800725
S315080084D007D5DFF8C0110A6832F0F002A068024337
S315080084E00A602078C00754D56068012806D1DFF8ED
S315080084F0A0010068800310D401207FE0606802288C
S3150800850005D163480068800107D4012076E06048F9
S315080085100068800701D4012070E05E4F3968890839
S31508008520890060680143396000F0D2F880466068C7
S3150800853001280ED1386810F00C00042829D000F064
S31508008540C7F8B0EB080041F289318842F2D303201C
S3150800855054E0606802280ED1386810F00C0008282C
S3150800856017D000F0B5F8B0EB080041F2893188421F
S31508008570F2D3032042E0386810F00C0F09D000F05F
S31508008580A7F8B0EB080041F289318842F3D30320FB
S3150800859034E0306810F0070085420BD23068C00816
S315080085A0C00028433060306810F00700A84201D0A8
S315080085B0012023E02078400706D536490A6832F4B8
S315080085C0E062E06802430A602078000707D5314870
S315080085D0016831F46051226951EAC201016000F074
S315080085E00FF837492B4A1268C2F30312895CC84050
S315080085F02A490860002000F071F80020BDE8F081E3
S3150800860000B585B001A82F49102200F08DF82E4834
S315080086100088ADF80000002000200020002000207F
S315080086201C4A116811F00C00042802D0082802D050
S3150800863014E0194813E001A8C1F38343C05CC903D9
S3150800864009D569461268C2F340428A5C1249484312
S31508008650B0FBF2F001E01D49484300E00E4805B0C2
S3150800866000BD0E480068704781B00C490968C90802
S315080086704FF47A72B1FBF2F14843009000BF0098BC
S31508008680411E00910028F9D101B070470000000092
S31508008690001002400410024000127A000400002074
S315080086A02410024080044242000042421C1002404C
S315080086B00070004020100240600042420020024044
S315080086C0508E0008408E0008AE87000800093D005D
S315080086D001480068704700BF0C00002010B5040070
S315080086E04FF47A700D490978B0FBF1F00C49096826
S315080086F0B1FBF0F000F0CAF8002801D001200CE028
S31508008700102C09D2002221005FF0FF3000F0ADF8EE
S3150800871004480460002000E0012010BD100000207D
S315080087200400002000000020103A07D330B4B1E856
S315080087303810103AA0E83810F9D230BC530724BFD5
S31508008740B1E80810A0E8081044BF51F8043B40F807
S31508008750043BD20724BF31F8022B20F8022B44BF72
S315080087600B7803707047121F17D35B0009D151F8B5
S31508008770043B20F8023B1B0C121F20F8023BF6D2E2
S315080087800BE051F8043B00F8013B1B0A20F8023BBA
S315080087901B0C121F00F8013BF3D238BF121D521EE4
S315080087A024BF11F8013B00F8013BF8D870470102D5
S315080087B010F007003E4B1A684FF6FF010A403D4984
S315080087C051EA00210A431A60704739480068C0F325
S315080087D002207047020052B2002A08D50901364A1B
S315080087E040B210F00F00104400F8041C03E0090121
S315080087F0324A40B21154704710B410F00700D0F155
S315080088000703052B01D3042301E0D0F10703041D58
S31508008810072C01D2002000E0C01E012414FA03F33D
S315080088205B1E1940814014FA00F0401E10400843B0
S3150800883010BC704780B5411EB1F1807F01D301207D
S315080088400EE0401E1E4908600F215FF0FF30FFF75B
S31508008850C1FF00201B49086007201B49086000204B
S3150800886002BD80B5FFF7A4FF01BD70B504000D0079
S3150800887016000020FFF7A9FF32002900FFF7BCFF0A
S315080088800100200040B2FFF7A5FF70BD80B5FFF7D5
S31508008890D1FF02BD042805D10B48016851F0040137
S315080088A0016004E00848016831F00401016070477E
S315080088B00CED00E00000FA0518ED00E000E400E029
S315080088C014E000E018E000E010E000E080B500F0F9
S315080088D001F801BD70470000F8B50200002000202D
S315080088E0002000250020002314E0DFF8B401066804
S315080088F036EA040404600CE0DFF8A8010668A6431B
S31508008900066048688002F0D5DFF8940106683443AB
S3150800891004605B1C102B80F0B88001269E400C6812
S315080089203440B442F5D14868002827D001281AD027
S3150800893002281DD003282FD0112816D012281AD0A5
S31508008940594FB8421AD0594FB84217D0584FB84263
S3150800895014D0584FB84211D0574FB8420ED0574F7F
S31508008960B8420BD01AE0CD6818E0CD682D1D15E089
S31508008970CD68083512E0CD680C350FE08868002808
S3150800898001D1042507E08868012802D10825166167
S3150800899001E00825566101E00025FFE7B4F5807F70
S315080089A001D2170000E0171DB4F5807F02D25FEAF6
S315080089B0830C03E0B3F1080C5FEA8C0C0F26D7F89A
S315080089C000E016FA0CF03EEA000E15FA0CFC5CEA1A
S315080089D00E0CC7F800C04868C0009AD53848076822
S315080089E057F001070760006810F001000090009832
S315080089F0344F1800800857F820C013F00300C0B29F
S31508008A00800086403CEA060C2F48824201D10026A7
S31508008A100FE02E48824201D101260AE02C48824204
S31508008A2001D1022605E02B48824201D1032600E047
S31508008A30042613F00300C0B28000864056EA0C0CE8
S31508008A401800800847F820C04868C00304D52248A3
S31508008A5006682643066003E01F480668A6430660C4
S31508008A604868800304D51D4806682643066003E067
S31508008A701A480668A64306604868C0027FF53CAFF8
S31508008A8008480668264306603BE7F1BDD2B2002ACD
S31508008A9002D089B2016102E089B209040161704716
S31508008AA00C040140080401400000111000001210D7
S31508008AB000002110000022100000311000003210C2
S31508008AC0181002400800014000080140000C01404F
S31508008AD00010014000140140000401400404014054
S31508008AE080B500F007F800F0ADF800F0B4F800F033
S31508008AF0AAF8FAE780B500F009F800F0D1F800F016
S31508008B0009F800F0DFF800F09FF801BD4848494928
S31508008B100860704700B58FB0012005905FF480307B
S31508008B200690002107910121099102210C910D90CF
S31508008B305FF4E0100E9005A8FFF7DAFA002800D0D7
S31508008B40FEE70F20009002200190002002904FF4CB
S31508008B50806003900020049002216846FFF79EFC7F
S31508008B60002800D0FEE70FB000BD00B585B032483A
S31508008B70016851F001010160016811F001010091DD
S31508008B8000992E490A6852F080520A60096811F065
S31508008B90805100910099016851F004010160016853
S31508008BA011F0040100910099016851F00801016073
S31508008BB0006810F00800009000980320FFF751FEA7
S31508008BC0002200217FF00B00FFF74FFE0022002154
S31508008BD07FF00A00FFF749FE002200217FF0090016
S31508008BE0FFF743FE002200217FF00400FFF73DFE59
S31508008BF0002200217FF00300FFF737FE0022002144
S31508008C007FF00100FFF731FE002200215FF0FF3000
S31508008C10FFF72BFE202001900120029000200390F0
S31508008C200220049001A90648FFF756FE05B000BDCC
S31508008C300080000808ED00E0181002401C100240F1
S31508008C40000801407047704780B50022202111486E
S31508008C50FFF71CFF01BD38B500F047F804000E4DBC
S31508008C602868201AB0F5FA7F13D30C49087800282B
S31508008C7007D101200870012220210648FFF706FFC8
S31508008C8006E000200870002220210248FFF7FEFEB9
S31508008C902C6031BD000801400800002011000020AA
S31508008CA080B50748016851F0100101600320FFF7FD
S31508008CB0D8FD0020FFF712FDFFF757FF002002BD81
S31508008CC00020024080B5FFF7CCFC4FF47A71B0FB68
S31508008CD0F1F0FFF7DBFD0420FFF7DCFD00220021A1
S31508008CE05FF0FF30FFF7C1FD01BD80B5FFF7F0FC6F
S31508008CF002BD80B500F004F8FFF7E8FD01BD0000ED
S31508008D0003490A680348007882180A60704700BF5A
S31508008D100C000020100000200F49086850F00100E0
S31508008D2008600E4A13680E48034013600B680D4826
S31508008D3003400B60086830F480200860106830F43F
S31508008D40FE0010605FF41F00074908605FF00060CE
S31508008D5006490860704700000010024004100240EF
S31508008D600000FFF8FFFFF6FE0810024008ED00E0DD
S31508008D7030B5016884684218416802EB5103C90797
S31508008D8003D54C4401E0491C05D19A420AD012F990
S31508008D90011B12F8015B002904F8015BF3D4491E94
S31508008DA0F7D5F2E70C3030BD10B5074979441831CC
S31508008DB0064C7C44163404E00A68081D11448847AA
S31508008DC00146A142F8D110BD0800000014000000B9
S31508008DD0A1FFFFFF640100001A0000000000002048
S31508008DE000F00DF8002801D0FFF7DEFFAFF3008092
S31508008DF00020AFF30080FFF773FE00F002F80120B1
S31508008E00704700F001B800000746384600F002F83F
S31508008E10FBE7000080B5AFF30080024A1100182076
S31508008E20ABBEFBE72600020002488546024880479B
S31508008E300248004718080020198D0008618E0008AE
S31508008E4002030405060708090A0B0C0D0E0F10107D
S31508008E5000000000000000000102030406070809DC
S31508008E60AFF30080AFF30080FFF7BAFFFFF7FEBF4E
S31508008E70FFF7FEBFFFF7FEBFFFF7FEBFFFF7FEBF18
S31508008E80FFF7FEBFFFF7FEBFFFF7FEBFFFF7FEBF08
S31508008E90FFF7FEBFFFF7FEBFFFF7FEBFFFF7FEBFF8
S31508008EA0FFF7FEBFFFF7FEBFFFF7FEBFFFF7FEBFE8
S31508008EB0FFF7FEBFFFF7FEBFFFF7FEBFFFF7FEBFD8
S31508008EC0FFF7FEBFFFF7FEBFFFF7FEBFFFF7FEBFC8
S31508008ED0FFF7FEBFFFF7FEBFFFF7FEBFFFF7FEBFB8
S31508008EE0FFF7FEBFFFF7FEBFFFF7FEBFFFF7FEBFA8
S31508008EF0FFF7FEBFFFF7FEBFFFF7FEBFFFF7FEBF98
S31508008F00FFF7FEBFFFF7FEBFFFF7FEBFFFF7FEBF87
S31508008F10FFF7FEBFFFF7FEBFFFF7FEBFFFF7FEBF77
S31508008F20FFF7FEBFFFF7FEBFFFF7FEBFFFF7FEBF67
S31508008F30FFF7FEBFFFF7FEBF0010FC0002A24A04BF
S30A08008F40F80001010024
S70508008E6103
